:10000000CD28A000FF3A8417800529082A04031987
:10001000C928BB208413200880060E280000102861
:10002000A90A0319AA0F0D288006C92883169B0068
:1000300083161C141A089B0AC92883169A001C15DB
:1000400055309D00AA309D009C149C1825281C1139
:100050009B0AC9280F39AF000310AF0DAF0D1F0861
:10006000E0392F0401389F00643071209F149F18DD
:1000700037281E08B30083161E088312B200C92851
:100080000830AF002418AC2021088400220824196D
:10009000C120241DC3202008840023098417800563
:1000A00020088400AA0CA90C00082304031C2306C2
:1000B00080005D20AF0B5028C92821088400220849
:1000C0008006000080060800AC01AB00FF30AB07E3
:1000D000031CAC07031CC9280330AA00DF307220C0
:1000E0006628AA01E83EA900AA09FC30031C7B2867
:1000F000A90703187828A9070000AA0F782829184B
:100100008128A91C8528000085280800013EB00030
:100110000A30AB00AC019020B00B8B282D080800F2
:10012000AE01AD011030AF002A0DAD0DAE0D2B08A4
:10013000AD022C08031C2C0FAE020318A6282B08B6
:10014000AD072C0803182C0FAE070310A90DAA0D3C
:10015000AF0B942829080800AB01AC01B328AA0C06
:10016000A90CAB0DAC0DFF3E0318AF282C08AA005C
:100170002B08A900C928A909AA09A90A0319AA0ACA
:1001800008008004C628FF3A8005C728FF3A841774
:10019000800583138312031308008301073099003D
:1001A00083169101903083129F00303083169F0098
:1001B000103091002F308500831285012130831685
:1001C000870083128701B701B601BB01BA01003075
:1001D0001620B8001820B90002301620C2001820DE
:1001E000C300C501C401C701C601C901C80103306C
:1001F000AC00E830652004302A20BA003308BB0088
:100200000310BB0CBA0C9D22BB08031D0E294630FF
:100210003A0203180E29B60A0319B70AC408031DC7
:100220001429C50803191829C403440A0319C5036E
:1002300045084404031D25293B08BD003A08BC00BD
:10024000C901C801C701C6012B293908BD003808FA
:10025000BC006430642044034504031D3F29831619
:100260009B01831238081D2039081D200230831697
:100270009B00831242081D2043081D203F29EB21CB
:10028000051C4B29C8306420C60A0319C70AC501DA
:100290000A30C400C421851C5629C8306420C80A0D
:1002A0000319C90AC5010A30C400D721051D6029F8
:1002B000C8306420C20A0319C30AC5010A30C40049
:1002C000C308031D672909304202031C6929C301C1
:1002D000C20101303902031C7629031D7329C33082
:1002E0003802031C7629B9016430B80007303702A0
:1002F000031C8D29031D8029D1303602031C8D2952
:100300000730B700D030B600B901B801C3010830DA
:10031000C200C5010A30C4008D29851E9129B7018C
:10032000B6019321FB280310420DB200430DB30028
:10033000B401B40DB50132083802A5003908A60091
:100340003308031C330FA602A7013408031C340F23
:10035000A702A8013508031C350FA802A81BC22953
:10036000A808031DC029A708031DC0293B082602B1
:10037000031CC229031DC02925083A020318C229FB
:100380000716C32907120800C708031DCB290B3025
:100390004602031CD3290A30B8070318B90AC7015B
:1003A0000A30C600D629B80A0319B90A0800C908D4
:1003B000031DDE290B304802031CE6290A30B8026F
:1003C000031CB903C9010A30C800EA29B803380A76
:1003D0000319B90308003D08AA003C08A900003031
:1003E0008620CA0070220730A0000430A300073026
:1003F000A1000230A2000130A4000830A900402072
:100400004B08A9004020AA010130A9000730840050
:1004100008300120013064203D08AA003C08A900F2
:1004200001308620CA0070220730A0000430A300EB
:100430000730A1000230A2000130A4000430A9005E
:1004400040204B08A9004020AA010130A900073034
:10045000840008300120013064203D08AA003C08D7
:10046000A90002308620CA0070220730A0000430A4
:10047000A3000730A1000230A2000130A400023026
:10048000A90040204B08A9004020AA010130A90082
:100490000730840008300120013064204308AA009E
:1004A0004208A90000308620CA0088220730A00038
:1004B0000430A3000730A1000230A2000130A400E4
:1004C0001030A90040204B08A9004020AA010130AB
:1004D000A9000730840008300120013064200800A2
:1004E0004A080B3C031C872A7722CB00872A02305C
:1004F0008A004A088207C034F934A434B0349934ED
:1005000092348234F83480349034BF34FF3408009D
:100510004A08083C031C9C2A8F22CB009C2A0230EC
:100520008A004A088207FF34FD34FC34DC349C34F2
:100530009834183410340034080001303B022C3059
:1005400003193A020318C82ABF01FA30BE00C101DC
:10055000C001C108031DC72A063040020318C72A7C
:100560003F083B02031CBA2A031DBE2A3E083A027A
:100570000318BE2ABA033A0A0319BB033230BE027B
:10058000031CBF03C00A0319C10A031DA92AEC2AD0
:100590000130BF00F430BE00C101C001C108031D1D
:1005A000EC2A043040020318EC2A3B083F02031CEB
:1005B000DF2A031DE32A3A083E020318E32ABA039E
:1005C0003A0A0319BB033230BE02031CBF03C00A40
:1005D0000319C10A031DCE2A08006300ED2AEF2A81
:02400E00A43FCD
:00000001FF
